:020000020000FC
:100000000FC022C130C132C132C132C12DC12DC198
:0400100031C12FC10A
:10002000F894F0E0E0E600E00193E03AE9F70EE949
:100030000DBF00E810E006BD16BD00E00BBF00E0FC
:1000400009BF00E005BB00E60ABF0EE008BF02E200
:1000500008BB01E007BB02E005BF00E00FBD00E008
:1000600003BF06E406BF00E009BD00E008BD00E2F2
:1000700007B900E003B907E006B90CE104BB00E8EA
:1000800008B9A89504B7077F04BF01B5006101BD99
:100090000EE401BD00E40BBF00E009BF09E1B02E92
:1000A00000E0A02E09E1D02E00E0C02E06E0302EA8
:1000B00000E4202E01E0502E0FEF402E01E0702EC4
:1000C0000FEF602E01E0902E0FEF802E90E07894DD
:1000D000A89590FFFDCF9E7F07E006B901E007B924
:1000E00007EC06B906B106FDFDCF44B055B007E0F8
:1000F00006B902E007B907EC06B906B106FDFDCF67
:1001000064B075B007E006B903E007B907EC06B9BB
:1001100006B106FDFDCF84B095B0132D022D000F62
:10012000111F000F111F512F402F042D152D31E0ED
:100130002FEF021B130B040F151FD12EC02E172DEE
:10014000062D1695079516950795572D462D400FA8
:10015000511F1D2D0C2D39E120E0021B130B352FF3
:10016000242F89D04AE036952795179507954A950B
:10017000D1F739E120E0020F131FD12EC02E06B3B4
:1001800005FD12C01D2D0C2D39E120E0021B130BC3
:100190000095109520E00894021F121F39E120E01D
:1001A000020F131FD12EC02E192D082D169507955D
:1001B000169507950F3F08F035C0F3E0E0E0E00F3B
:1001C000F11FC8951D2D0C2D3B2D2A2D021B130B45
:1001D00059F108F412C030E0202D021B130B08F473
:1001E00009C01B2D0A2D30E0202D020F131FB12E48
:1001F000A02E1AC0BD2CAC2C17C01095009520E085
:100200000894021F121F30E0202D021B130B08F46C
:1002100009C01B2D0A2D30E0202D021B130BB12E1F
:10022000A02E02C0BD2CAC2CDB2DCA2DD695C795B7
:10023000D695C795C09A000000000000000000009D
:100240002197C9F7C09844CFFFB6B0E0A0E006B34D
:1002500001FD04C01196B4FD04C0F9CF3B2E2A2E37
:100260009160FFBE189518951895189518951895D2
:100270001895189518954F935F936F9366274427A9
:1002800011232AF4439500951095061F161F33235A
:100290002AF4439520953095261F361F40FB0FD03A
:1002A00046F40095109540955095061F161F461F61
:1002B000561F242F352F6F915F914F910895551B35
:1002C000441B61E110F4420F531F57954795179552
:0802D00007956A95B9F708953E
:100300000606060606060606070707070707070785
:100310000707070707080808080808080808080862
:1003200009090909090909090909090A0A0A0A0A38
:100330000A0A0A0A0B0B0B0B0B0B0B0B0C0C0C0C0D
:100340000C0C0C0C0D0D0D0D0D0D0D0E0E0E0E0EDC
:100350000E0F0F0F0F0F0F0F1010101010111111A3
:100360001111111212121212131313131314141465
:10037000141515151515161616161617171718181D
:1003800018181919191A1A1A1A1B1B1B1C1C1C1DC8
:100390001D1D1D1E1E1E1F1F1F2020212121222268
:1003A00022232323242425252526262727282828F9
:1003B00029292A2A2B2B2C2C2D2D2E2E2F2F303075
:1003C00031313232333334353536363737383939DF
:1003D0003A3B3B3C3C3D3E3F3F404141424343442E
:1003E0004546464748494A4A4B4C4D4E4F4F50515F
:1003F00052535455565758595A5B5C5D5E5F606165
:00000001FF
